:100000008DC00000A6C00000A4C00000A2C0000077
:10001000A0C000009EC000009CC000009AC000006C
:1000200098C0000096C0000094C00000D7C3000034
:1000300090C000008EC000008CC000008AC000008C
:1000400088C0000086C0000084C0000082C000009C
:1000500080C000007EC000007CC0000030C10000F5
:1000600078C0000076C0000074C0000072C00000BC
:1000700070C0000022034100720064007500690036
:100080006E006F0020004A006F007900730074005A
:10009000690063006B0000001003410072006400FF
:1000A000750069006E006F00000004030904090276
:1000B0002200010100C03209040000010300000019
:1000C000092111010001223A000705810308000AF5
:1000D0001201100100000008EB03432000000102A0
:1000E000000105010904A1010901A1000501093070
:1000F000093109320933093409350936093716003F
:100100008026FF7F751095088182C0050919012995
:100110002815002501750195288102C011241FBEF4
:10012000CFEFD2E0DEBFCDBF11E0A0E0B1E0EAE763
:10013000FFE002C005900D92AE30B107D9F711E093
:10014000AEE0B1E001C01D92A83CB107E1F72CD0B0
:1001500012C756CFCF93DF9384B7877F84BF28E140
:100160000FB6F89420936000109260000FBE80E1FB
:1001700090E09093CD008093CC0086E08093CA00FD
:1001800082E08093C800C9ECD0E02883539A5A9A41
:100190008AB180638AB98BB180638BB914D388E943
:1001A0008883DF91CF910895D5DF2FB7F8948AE344
:1001B00091E09093B9018093B8019093BB01809333
:1001C000BA012FBF789480E091E00AD6B5D480912F
:1001D0000E0190910F01892BB1F380910E01909146
:1001E0000F01019790930F0180930E0180910E01F2
:1001F00090910F01892B39F75D9AE5CF0895089505
:1002000080E091E0CAD5E2EEF0E0808184608083F6
:10021000089580E091E0A1C480910B0190910C01C0
:10022000009729F0019790930C0180930B0108959A
:100230000F931F93CF93DF939FB7F8948091BC01E6
:100240009FBF853140F1C0E1D1E08AE391E0E091C8
:10025000BA01F091BB015191F093BB01E093BA0157
:10026000E85BF14021F49093BB018093BA016FB732
:10027000F8944091BC0141504093BC016FBF599329
:10028000E1E0C532DE0719F75D9880ED97E09093C5
:100290000F0180930E0185E1E0E1F1E0D9010190C9
:1002A0000D928A95E1F785E190E0F80191838083D2
:1002B00080E0DF91CF911F910F91089508951F92D3
:1002C0000F920FB60F9211242F938F939F93EF935A
:1002D000FF938091CE009EB3943029F52FB7F89408
:1002E0009091BC012FBF9E37F1F0E091B801F091E1
:1002F000B9018083E091B801F091B901CF01019675
:100300009093B9018093B801885B914021F48AE30E
:1003100091E0928381839FB7F8948091BC018F5FB5
:100320008093BC019FBFFF91EF919F918F912F917F
:100330000F900FBE0F901F901895292F3327233051
:100340003105B1F04CF42130310509F439C02230C7
:10035000310509F03AC007C02132310539F12232A6
:10036000310549F132C0E2E2F0E08EEA90E031C0BE
:1003700099278130910561F08230910581F0892BB8
:1003800021F5EAEAF0E0E491F0E08AEA90E021C0A9
:10039000E8E9F0E0E491F0E088E990E01AC0E4E7F1
:1003A000F0E0E491F0E084E790E013C0E9E0F0E0F1
:1003B00080EC90E00EC0EAE3F0E082EE90E009C04D
:1003C000E2E1F0E080ED90E004C0E0E0F0E080E009
:1003D00090E0DA018D939C93CF01089528E030E0FE
:1003E00040E003C04F5F220F331F28173907D0F3B7
:1003F000842F8295807F08958093E900EBEEF0E0F2
:10040000808181608083EDEEF0E010826093EC00EB
:1004100040838091EE00881F8827881F08951092DE
:10042000F40080E08093E9001092F0001092E80060
:100430001092ED009091EB009E7F9093EB008F5F08
:10044000853081F708958091C00187FD05C08091B6
:10045000E80080FF0DC010C08091E80082FD04C05C
:100460008EB38111F9CF08958091E8008B7707C092
:100470008EB38111ECCF08958091E8008E77809340
:10048000E800089585E69091EC0090FF05C09091FA
:10049000E80090FF05C01BC09091E80092FD17C0D6
:1004A0009EB39923B1F09EB39530A9F09091EB00E3
:1004B00095FD13C09091E10092FFE5CF9091E1008E
:1004C0009B7F9093E1008150F1F684E0089580E0F5
:1004D000089582E0089583E0089581E00895AF9241
:1004E000BF92CF92DF92EF92FF920F931F93CF9321
:1004F000DF931F92CDB7DEB7C82E8B017A019983A7
:10050000C1DFD82E9981811127C0AC2CB92E1CC017
:100510008091E80085FD11C08091E8008E7780937E
:10052000E800E114F10421F4ADDF882369F010C084
:10053000F70109958130C1F70DC0F50181915F0187
:100540008093F100015011090115110509F704C04C
:10055000D82E02C075E0D72E8D2D0F90DF91CF9150
:100560001F910F91FF90EF90DF90CF90BF90AF90D1
:1005700008952091C6013091C7012617370748F02A
:100580006115710539F42091E8002E772093E80079
:1005900001C0B901FC0190E029C08091E80083FD11
:1005A00037C08091E80082FD2DC08EB3882391F181
:1005B0008EB3853089F18091E80080FF17C080916B
:1005C000F20006C091919093F100615071098F5F24
:1005D0006115710511F08830A8F391E0883009F0B9
:1005E00090E08091E8008E778093E80061157105B6
:1005F000A1F69111D2CF06C08EB3882359F08EB3E5
:10060000853051F08091E80082FFF6CF80E00895B8
:1006100081E0089582E0089583E008952091C60165
:100620003091C7012617370748F06115710539F475
:100630002091E8002E772093E80001C0B9019C01C9
:1006400090E02CC08091E80083FD3AC08091E800E2
:1006500082FD30C08EB38823A9F18EB38530A1F11D
:100660008091E80080FF1AC08091F20009C0F90172
:100670002F5F3F4FE491E093F100615071098F5F6C
:100680006115710511F0883090F391E0883009F020
:1006900090E08091E8008E778093E8006115710505
:1006A00089F69111CFCF06C08EB3882359F08EB34F
:1006B000853051F08091E80082FFF6CF80E0089508
:1006C00081E0089582E0089583E008956115710541
:1006D00029F42091E8002B772093E8009C0121C0A9
:1006E0008091E80083FD2BC08EB3882371F18EB317
:1006F000853039F18091E80082FFF2CFF90107C01F
:100700008091F10081939F016150710929F09F014F
:100710008091F2008111F4CF8091E8008B77809373
:10072000E80061157105E1F68091E80080FD0BC0DD
:100730008EB3882351F08EB38530B1F702C081E0CB
:10074000089583E0089580E0089582E0089540D000
:1007500042D01EBA1092BE011092BD0184E089BD44
:1007600089B5826089BD09B400FEFDCF8091D800B3
:10077000982F9F779093D80080688093D8008091BD
:1007800063008E7F809363008091D8008F7D80937B
:10079000D8008091E0008E7F8093E0008091E1009E
:1007A0008E7F8093E1008091E20081608093E2007F
:1007B0008091E100877F8093E1008091E200886072
:1007C0008093E2000895C3DF81E08093BF01089524
:1007D0001092E20008951092E10008951F920F9286
:1007E0000FB60F9211242F933F934F935F936F9304
:1007F0007F938F939F93AF93BF93EF93FF938091DA
:10080000E10080FF1BC08091E20080FF17C0809153
:10081000E1008E7F8093E1008091E2008E7F8093E3
:10082000E2008091E20080618093E2008091D80034
:1008300080628093D80019BC1EBAE1DC8091E1008F
:1008400084FF29C08091E20084FF25C084E089BD37
:1008500089B5826089BD09B400FEFDCF8091D800C2
:100860008F7D8093D8008091E1008F7E8093E1009E
:100870008091E2008F7E8093E2008091E2008160AF
:100880008093E2008091BE01882311F084E001C0D2
:1008900081E08EBBB3DC8091E10083FF22C08091B8
:1008A000E20083FF1EC08091E100877F8093E1001A
:1008B00082E08EBB1092BE018091E1008E7F80931A
:1008C000E1008091E2008E7F8093E2008091E2005F
:1008D00080618093E200A3DD42E060E080E08CDD97
:1008E0002AD18091E10082FF0AC08091E20082FF5C
:1008F00006C08091E1008B7F8093E1008DDCFF9149
:10090000EF91BF91AF919F918F917F916F915F9187
:100910004F913F912F910F900FBE0F901F90189500
:100920000F931F93CF93DF9300D0CDB7DEB7E0ECEA
:10093000F1E08091F100819381E0E83CF807C9F78C
:100940008091C0019091C101953009F472C038F4D2
:10095000913089F170F0933009F0E4C02CC09830E8
:1009600009F4A8C0993009F4B7C0963009F0DAC08C
:1009700082C0803821F0823809F0D4C003C0909141
:10098000BD010FC08091C4019091C5018770992766
:100990008093E9009091EB0095FB992790F91092D4
:1009A000E9008091E800877F8093E8009093F10050
:1009B0001092F1008AC0882319F0823009F0B2C089
:1009C0008F71823009F09FC08091C20181112BC0CC
:1009D0008091C4019091C50187709927009709F40F
:1009E00092C08093E9002091EB0020FF8CC0209101
:1009F000C101233021F48091EB00806212C09091FC
:100A0000EB0090619093EB0021E030E001C0220FF9
:100A10008A95EAF72093EA001092EA008091EB00B1
:100A200088608093EB001092E9008091E800877F56
:100A30004FC0811177C00091C2011091C301809114
:100A4000E800877F8093E800FEDC04C08EB3882333
:100A500009F459C08091E80080FFF8CFC8018F7772
:100A60009927009711F023E001C022E02EBB806897
:100A70008093E30048C08058823008F053C0AE0134
:100A80004F5F5F4F6091C4018091C2019091C3019B
:100A900054DC0097C1F12091E800277F2093E80003
:100AA000BC0189819A81BADD8091E8008B778093BF
:100AB000E80029C08038B1F58091E800877F8093F5
:100AC000E8008091BE018093F1008091E8008E776C
:100AD0008093E800B8DC17C0811124C09091C20156
:100AE000923088F48091E800877F8093E8009093AB
:100AF000BE01A9DC8091BE01882311F084E001C011
:100B000083E08EBB7DDB8091E80083FF0DC0809188
:100B1000EB0080628093EB008091E800877F8093F8
:100B2000E80002C076DBEFCF0F900F90DF91CF91FE
:100B30001F910F9108950895CF938EB3882359F094
:100B4000C091E900C7701092E9008091E80083FD30
:100B5000E7DEC093E900CF9108956F927F928F9264
:100B60009F92AF92BF92CF92DF92EF92FF920F933C
:100B70001F93CF93DF9300D01F92CDB7DEB77C01D8
:100B8000ADB6BEB68091E80083FFF0C0F70180816A
:100B900090E02091C4013091C5012817390709F070
:100BA000E5C08091C101833009F492C030F48130F6
:100BB00071F0823009F0DAC0C1C08A3009F4A7C0F0
:100BC0008B3009F492C0893009F0D0C049C08091BF
:100BD000C001813A09F0CAC08DB69EB68091E80086
:100BE000877F8093E8001A8219828091C201109158
:100BF000C3018B83F70147818DB79EB7841B910991
:100C00000FB6F8949EBF0FBE8DBFCDB6DEB6EFEF28
:100C1000CE1ADE0A360150E060E070E0C601A4D1D1
:100C2000412F41508E010F5F1F4F9601BE016D5F36
:100C30007F4FC701FDDAF701258136812115310586
:100C400029F0478150E0B601C90185D11092E90031
:100C500069817A81C3018DDC8091E8008B772EC099
:100C60008091C001813209F081C08DB69EB680911D
:100C7000E800877F8093E8000091C6011091C701CA
:100C80007090C2016090C3018DB79EB7801B910B1D
:100C90000FB6F8949EBF0FBE8DBFCDB6DEB6EFEF98
:100CA000CE1ADE0AB801C60111DD462D415096016B
:100CB000672DC70103DB8091E8008E778093E80001
:100CC000882D992D0FB6F8949EBF0FBE8DBF4EC0D4
:100CD0008091C001813A09F049C08091E800877F86
:100CE0008093E800F701808539C08091C00181328E
:100CF000E9F58091E800877F8093E8009091C20138
:100D000081E0911101C080E0F70180872EC08091C1
:100D1000C001813259F58091E800877F8093E80017
:100D20008091C2019091C301882736E096958795FE
:100D30003A95E1F7F7019287818717C08091C0014A
:100D4000813AA1F48091E800877F8093E800F70161
:100D50008185928596958795969587958093F100E4
:100D60008091E8008E778093E8006DDB0FB6F894F1
:100D7000BEBE0FBEADBE0F900F900F90DF91CF9112
:100D80001F910F91FF90EF90DF90CF90BF90AF90A9
:100D90009F908F907F906F900895CF93DF93FC0189
:100DA0000896DC0185E0ED0119928A95E9F781E06A
:100DB000808784EF91E092878187228133818481CB
:100DC000882311F0C4E001C0C0E0D181C90106DB75
:100DD0004C2F482B426061EC8D2FDF91CF910CCBD3
:100DE0004F925F926F927F928F929F92AF92BF923B
:100DF000CF92DF92EF92FF920F931F93CF93DF93E7
:100E000000D01F92CDB7DEB77C01ADB6BEB68EB3B3
:100E1000843009F07AC0F70181818093E9008091E4
:100E2000E80085FF72C06DB67EB647818DB79EB76C
:100E3000841B91090FB6F8949EBF0FBE8DBFCDB62F
:100E4000DEB6EFEFCE1ADE0A1B821A821982460145
:100E500050E060E070E0C60187D08E010F5F1F4F49
:100E6000960140E0BE016D5F7F4FC701E1D9482E7A
:100E7000F70121853285232B31F001E010E0238535
:100E80003485232B11F000E010E0F701C580D680F7
:100E9000C114D10489F049815A81B601C4014ED0F0
:100EA00055245394009709F4512CF701478150E0E1
:100EB000B401C60150D001C0512C29813A81232BA5
:100EC000E9F0411004C0511002C000FF17C0F70143
:100ED000218532853487238781818093E9008B8146
:100EE00081118093F10069817A8140E050E0C40172
:100EF000F6DA8091E8008E778093E800862D972DB2
:100F00000FB6F8949EBF0FBE8DBF0FB6F894BEBE4D
:100F10000FBEADBE0F900F900F90DF91CF911F913C
:100F20000F91FF90EF90DF90CF90BF90AF909F9088
:100F30008F907F906F905F904F900895FB01DC0140
:100F400004C08D910190801921F441505040C8F7A0
:100F5000881B990B0895FB01DC0102C001900D92E2
:100F600041505040D8F70895DC0101C06D934150C5
:0A0F70005040E0F70895F894FFCF19
:0E0F7A00000108000025011500000000000025
:00000001FF
